:10000000272800000000000009000900090009007D
:1000100000309300FF3085008511861F1314061FE2
:10002000931785150511861F9314061F13170515C1
:100030008510861F1315061F931685140510861F3D
:100040009315061F1316AF2013080800003485010E
:1000500086018316003065008B138B01C230660069
:100060007F308100811383129101AD01163084002D
:10007000C620AF2086150030A700A800A900920076
:10008000203091000830AB00303084000611861C0F
:100090004E2800000000061586184628061186180E
:1000A0005628A70A00000615861C4E282708AA0015
:1000B0000310AA0C0830A600A901D820A90D2A080F
:1000C000A800061129108618291406150000A80B8F
:1000D00061282A08A80006110615A80B6B28A60B94
:1000E0005E280830A600290892008000840AF320C8
:1000F000AB0B7B2889280830A600A901D820D8207E
:10010000061106158618802806110615861C8428F7
:100110005D283030910006100830A6001630A70088
:100120003030A800270884000008A90028088400AF
:1001300000082902031DE128A70AA80AA60B922895
:100140000614B82005160A30A600A701A801A80BBE
:10015000A728A70BA728A60BA7280610E228851515
:10016000A6011030910019212602031985110800FB
:10017000A6011030910019212602031DC228FF306C
:100180008515C42800018511920005290820AD01BC
:10019000AC000310AC0DAD0DAC0DAD0DAC0DAD0D47
:1001A0001630840091015021E320F62050210800F0
:1001B0002708A800A80AA80A06110615A80BDC281B
:1001C0000800AF20E228083093002C0820210808FE
:1001D0008000840A392108088000840A930BEA28E9
:1001E0005029103091000521910A08001630840032
:1001F00008309300000892000521910A840A930BAD
:10020000FA2883168B1383120800831212088800C1
:1002100011088900831608128B13081555308900C0
:10022000AA30890088148B178818142908118312A2
:1002300008001108890083160814831208080800B2
:100240008900482103102B2109082E21482103147D
:100250002B21392108002D0D0F39A0388800C2301C
:100260006600342134216229372137213721880D56
:100270005C29D230660042214221901C0310901864
:1002800003105A294521452145216521880D080083
:100290000616C230660086160000061200005829B5
:1002A0000612C23066000000861600000616000026
:1002B00086120800C2306600031C061203180616D8
:1002C00086165729D2306600811386160000031463
:1002D000061E0310000058298316660083120800CA
:02400E00F93F78
:00000001FF
